:020000040000fa
:080000000002040000000000f2
:020000040000fa
:10040000efb42000007f24000001880000000000fd
:100410000c0007008081230001002000110007006c
:10042000000020000000e000020032000000020096
:1004300000000000a0360200000000000040da00ca
:100440000000fe004440a900e01620000000e0008b
:100450000300320000002000a00188004440a800f2
:100460000000060091018800800078000000eb0089
:1004700015003700e280400032a0b4009101ba00bc
:10048000e280400032a0b4009102ba00e280400055
:1004900032a0b4000002eb00472bde00f507b200eb
:1004a000602ce10004003a000059eb008301e900f0
:1004b000fdff3e00040037006128e100010032002a
:1004c0000082eb00040007001101ba000200e00006
:1004d000e8ff3a00000006003159ba008301e90044
:1004e0000c0032002159ba008301e90008003200f3
:1004f0000400e00003003a00e280400032a0b400b3
:10050000f5ff370011d9ba008301e900faff3a007c
:100510008100e800e180400032a0b4000000060045
:10052000bc2d040000000000cc2d040000000000e1
:10053000dc2d040000000000ec2d04000000000091
:10054000fc2d0400000000003c2e04000000000010
:10055000b02e0400000000007c2e0400000000000b
:10056000962e040000000000e003040000000000dc
:10057000ec874700889fbe008a9fbe008c9fbe000c
:100580008e1f7800f0b79f0081bf9f008204780023
:1005900000047800010037000804e80018477800dc
:1005a0000e00fb00b20007000000e000faff3a0076
:1005b000d0c2b300804f57000500320000c0e900f0
:1005c000804f5700020032000047780001003700da
:1005d0000804e8000900e00045003500e18f540000
:1005e0004300320040022000808f540040003c0055
:1005f0000900e0000e003400f08f54001a003a00a9
:1006000000c3b300984f100016003a0098409000c5
:1006100080c7b30080cf50000300320080c5b30014
:1006200080cf50000f003a000884e8000e00370029
:10063000a900200000c3b300984f10000a003a0040
:100640009840900080c7b30080cf50000400320073
:100650008900200080c5b30080cf500002003a001e
:100660000884e800090120000805780000c3b300f1
:10067000010037000a05e8009a4f1000fdff320024
:100680008a0578006066b8000e00370090a620004a
:1006900000425200c4ef9f006149b9000c00be0047
:1006a000af0907004fea97000401fb00cf91de007d
:1006b0008b05e800ccb79f00ddb79f000006410026
:1006c000818649001b00fb00710007008000780054
:1006d0000901780090a6200074000700000278004d
:1006e0000000e000e9ff3a008b0f540006003a00da
:1006f0000fb897000000e00029003200ffb097001b
:1007000001087800260037008a80550040a42000a8
:1007100060c07c000000fb00008050001600330029
:100720004240a9000f003c004fe997000200fb0087
:10073000cf80de000000560081805e00800f5600f2
:10074000818f5e00070039006149b9009a0a0700ed
:100750004fb19700dfb19700820f5000838f580090
:100760000500320020022000305a88000086eb008d
:100770008086eb0005003700d0c2b300804f5700e1
:1007800002003a0060061600e0861e008fb997004e
:100790000300e000030032008b09780001003700fd
:1007a0006066b8000c00be004f0778004f06be0020
:1007b0004f05be004f04be00cf00b1000000060090
:1007c000881f7800020478004800070008004000f5
:1007d0004f047800000006000000fa00881f78002f
:1007e000000478003fb99700ea8157008000780044
:1007f000003e200044000700800078000000e00078
:10080000020035000040eb0000f4780001007800a1
:100810004f0478000080fa00000006008000780095
:100820001106b100030035009101b10001003c0048
:100830000050a100000006000003b1000b003500cd
:100840009000b100080034008000b10007003500be
:100850009001b100040034007000b10003003500c5
:100860009001b10001003c001000050000000500ef
:100870006900e100040035006d00e1000300340070
:100880000002b10001003200000005001000050068
:10089000800078001104b100030035009101b1001f
:1008a00001003c000050a000000006008001eb00a9
:1008b000040037008301e80090cf100004003200ec
:1008c0000000e800828f5100faff3a000000eb00c0
:1008d00000000600205a80000000e0000100320005
:1008e0000000010060b42000000006008001eb0061
:1008f0000200370061f079008301e800828f510027
:10090000fcff3a00000006006200fa00889fbe006b
:100910008a9fbe000004be000205780083007800b4
:1009200060f92f000f004000b000070088979f007b
:1009300099979f000000eb00a09f9f009a457800c8
:100940000b80fb000000ea00cf04de0050c2b300c1
:1009500080cf550002003200090478000100370002
:100960000904e9000800e0000b0034001f90970024
:10097000080178008a0078008f9197000300010039
:1009800090979f000000e000930032002f9897009e
:1009900000004400a09f9f000905450050c2b3001d
:1009a00080cf5500040032000b04e000e3ff3a0062
:1009b0002f989700890037000000eb00809f9f0070
:1009c000f0979f00e0979f00d0979f00c0979f00ef
:1009d000b0979f00c09f9f000900370060b32000c0
:1009e0000080500000004000a1b22000e10078002b
:1009f0004f98970001007000c09f9f000a05e80013
:100a00001a4478008800fb0060b320007c000700d7
:100a1000800078000000e000f0ff3a00a0c2b300c0
:100a2000804f54000e003a00bf8897000180e90013
:100a3000b08f9f0010007800b09f9f000000e00082
:100a400005003d000000ea00b09f9f004f9897000e
:100a50000020a000c09f9f000a05e800100037009a
:100a6000b19f9f0003fd2f00f4ff2700080037000f
:100a70003f989700840f5000040032006a00b900cc
:100a80000000410003004000b09f9f000a05e800fd
:100a90001a01fb0003004100e90f5000f4ff36008b
:100aa000e0c2b3009a4f1000040032000080eb0057
:100ab000909f9f008a0478001c0037008a04e80099
:100ac000a0c2b300994f100007003a00bf889700fa
:100ad0000180e900b08f9f0010007800909f9f0078
:100ae0008a84e800110037000000eb00909f9f000f
:100af00003fd2f00f4ff2700080037001f98970020
:100b0000840f5000040032006a00b9000000410068
:100b100003004000909f9f008904e8001901fb003a
:100b200003004100e90f5000f4ff3600194478003b
:100b30008800fb00c0b32000310007000000e00087
:100b400002003a0000447800010037008904e80000
:100b5000a87f9f0080c6b300804f540004003a0075
:100b6000994f14000a003a00664050000600370012
:100b7000c0c6b300804f540005003a00994f1400de
:100b800003003a0065404000a07f9f008904e80010
:100b90000905e800c8fb2f000f04440060f92f008e
:100ba0000f0040008085e800880178001941780036
:100bb000800078000b007800e40007000000e000ef
:100bc00005003a00880078000b0078001500070047
:100bd0000000e00059ff3d000080eb004f05be0023
:100be0004f04be000080fa00000006000200fa0078
:100bf000f1bf9f00010878000080fa0000000600a5
:100c0000040037000204e00001003a000000050083
:100c10000000e80010417800814f5100f9ff3a00d0
:100c2000000006000400fa00889fbe008a9fbe00f4
:100c30008c1f78000004780001067800700890008e
:100c4000f80090000100500088089000010050005a
:100c50009808900001005000a80890000100500082
:100c6000b808900001005000c808900081055000ad
:100c70000002220090bf9f0000032300a0bf9f003e
:100c8000081090000028a30018003a000b00e000b4
:100c9000160034008b04780009057800e28f5400b8
:100ca000020036002a002000020037000900e000a0
:100cb0000b00340058009000c80190000a01780031
:100cc000ee80570003000100500498000000e0008f
:100cd000960032006808900000004500600c980003
:100ce0008a8454004240a900ebff3c007801900048
:100cf0000200e0000b00340058009000c801900092
:100d00008c00780003000100500498000000e0000f
:100d10008600320068089000f80090000100400052
:100d2000600c9800880c90000900e0001500340069
:100d300009057800e28f5400020036002a002000e6
:100d4000020037000900e0000b003400580090005a
:100d5000c80190000a017800ec80570003000100f0
:100d6000500498000000e000700032006808900015
:100d700000004500600c98008a8454004240a9009d
:100d8000ebff3c00180990000200e0000b0034006b
:100d9000e800900058009000c80190000300010096
:100da000500498000000e0006000320068089000e5
:100db0009808900001004000600c9800a80c90007a
:100dc0000900e0001500340009057800e28f5400a6
:100dd000020036002a002000020037000900e0006f
:100de0000b00340058009000c80190000a01780000
:100df000ec80570003000100500498000000e00060
:100e00004a0032006808900000004500600c98001d
:100e10008a8454004240a900ebff3c00380990004e
:100e20000200e0000d003400e80090001808900077
:100e30008080400058009000c8019000030001002d
:100e4000500498000000e00038003200680890006c
:100e5000b808900001004000600c9800c80c900099
:100e60000900e0001500340009057800e28f540005
:100e7000020036002a002000020037000900e000ce
:100e80000b00340058009000c80190000a0178005f
:100e9000ec80570003000100500498000000e000bf
:100ea000220032006808900000004500600c9800a5
:100eb0008a8454004240a900ebff3c0008109000d7
:100ec0000028a3001b0032000b00e00019003400d2
:100ed0008b04780009057800e28f54000200360088
:100ee0002a002000020037000900e0000b00340057
:100ef00058009000c80190000a017800ee80570069
:100f000003000100500498000000e00007003200d8
:100f10006808900000004500600c98008a84540026
:100f20004240a90003003400eaff37000080eb00d4
:100f3000010037000000eb004f0678004f05be00af
:100f40004f04be000080fa0000000600889fbe002b
:100f50008a1f78000004780001027800824478003b
:100f60000305780070c6b300804f510021003c009b
:100f700000c0e900804f5100de003d00724050008b
:100f8000804f51004b0132000d003c006c4050007e
:100f9000804f51005e013c0000c0e900804f5100cd
:100fa000d4003d0050c2b300804f510055013200c3
:100fb0007c404000804f510055013a00cd00370081
:100fc00010c6b300804f5100ca00320004003c003c
:100fd00069405000804f51004d013a0072003700c7
:100fe00030c6b300804f5100180032000040e800c6
:100ff0000900370000c7b300804f51001e013200c6
:1010000008003c0000c0e900804f5100e4003200bd
:1010100065003c006540500080cf54003c013a0020
:101020000f00370050c7b300804f51005e00320000
:1010300063404000804f51005b003200654050002b
:10104000804f510032013a001a0137009180e900c7
:10105000010a780078009000917178003201370021
:10106000a8609000c0c6b30080cf50000a003a00cc
:101070009400780064805000000a78001000be00e0
:101080004f89de00cf91de000002be00020378002f
:10109000820378001300370010c7b30080cf5000e0
:1010a00003003200a0c6b30080cf500006003a0013
:1010b0009400780068805000000a78003002be007a
:1010c0002003be00070037001480e900000a780002
:1010d0001000780000027800cfa2de00050378003f
:1010e00086037800049cbe000694be00a8609000b1
:1010f00080c6b30080cf50000e00320020c6b3007f
:1011000080cf500005003a000400fb00cf80de00d5
:1011100001017800820178000a00370040c7b3005f
:1011200080cf5000030032006640400080cf500066
:1011300006003a0004007800cf80de00010178004c
:1011400082017800009cbe000294be003800be0000
:101150002801be00e00f5000e08f5800e00f59005a
:10116000e08f590003003d0078009000d1c2b30029
:101170000a003700081090000018a3000300320096
:1011800078009000b1c2b300040037000008a3004b
:10119000530032007800900001c2b300017578005e
:1011a0000000e8004d003700a8609000c0c6b30002
:1011b00080cf500006003a00940078006480500010
:1011c000000a78001002be006033b8001300370038
:1011d00010c7b30080cf500003003200a0c6b30098
:1011e00080cf500006003a009400780068805000dc
:1011f000000a78003002be002003be00070037005e
:101200001480e900000a78001000780000027800dd
:10121000050020000600200007002000049cbe00fe
:101220000694be00a860900080c6b30080cf500036
:101230000e00320020c6b30080cf500005003a00f7
:101240000480fb00010020000200200003002000b9
:101250000a00370040c7b30080cf500003003200bf
:101260006640400080cf500006003a00040078003d
:10127000010020000200200003002000009cbe00ae
:101280000294be00081090000038a3001400320041
:101290003800be002801be00e00f5000e08f58006b
:1012a000e00f5900e08f59000d00320080c7b300f5
:1012b00080cf54000300320080c5b30080cf5400bb
:1012c00007003a007800900001c3b3000175780070
:1012d0008000e80009f578000080e80070049800bc
:1012e0007800900000004500600498008940780074
:1012f0006d003700a8609000c0c4b30080cf5000dc
:1013000006003a009400780068805000000a7800d7
:101310005001be004000be00050037009400780078
:1013200064805000000a78001000be00b207070079
:10133000009cbe000294be00380090000000e00057
:1013400003003d0078009000d1c2b3000a003700ce
:10135000081090000018a3000300320078009000ed
:10136000b1c2b300040037000008a300050032003a
:101370007800900001c2b300017578000000e80019
:101380007004980078009000000045006004980008
:101390008940780008007800f901070064003700f0
:1013a000a8609000c0c6b30080cf50002500320076
:1013b0000a003c006440500080cf500028003200fa
:1013c00000c0e80080cf5000140032006840500098
:1013d00080cf500022003a000a00370040c7b30017
:1013e00080cf50001e0032006640400080cf500089
:1013f0001b0032006940500080cf500018003a00b6
:10140000060037001480e900000a78001000780018
:10141000485c900008487800450037001480e900d7
:10142000000a78001002780068089000cf80de0083
:101430000101780082017800009abe000292be008d
:101440003b0037001480e900000a780010017800a2
:1014500068089000cf80de000089be0034003700ad
:101460001480e900000a780010007800680c9000f1
:10147000080878002e0037001180e9008008780005
:1014800010007800cf80de00010178008201780032
:10149000009cbe000294be00780090000000450051
:1014a0006004980081c7b30008007800240007009a
:1014b0001f0037001480e900000a7800100078004f
:1014c00060049800580990000200e00002003d000e
:1014d000a4010700090037008000eb00f3fc0700bf
:1014e000800078000000e0000300320068009000f7
:1014f000008050000100370058089000100c980040
:101500000b00370078009000027578000600370065
:1015100078009000800045000904e00001003a00d6
:1015200059c2b300894878000000e80070049800b0
:101530000000eb004f0578004f04be0000000600dd
:101540002f03b000889fbe008a9fbe008c9fbe0004
:101550008e1f78000007780090b12000c0b79f0070
:1015600080c5b30080cf50000800320082b0200058
:10157000c2b79f007740400080cf500003003a0080
:1015800083002000b3b79f000a00370080c7b30074
:1015900080cf500005003200a4002000b4b79f00a7
:1015a00080c5b30080cf500002003a000501200042
:1015b000b5b79f003e04be002e05be0040c6b30076
:1015c00080cf5000030032006540400080cf5000c3
:1015d0000b003a00e00f5400e08f5c00e00f5d006c
:1015e000e08f5d0006003d006000b8006011b800ab
:1015f00008045000898458000a0559008b85590059
:10160000bfb39700e88f530003003200f08f530000
:1016100045003a0002003700360020000100370084
:1016200046002000e00f5400e08f5c00e00f5d00fa
:10163000e08f5d0005003a005e0890008101200007
:10164000a1b79f000000e000080032003fb1970002
:101650000200e90008006000cfb197006340780005
:1016600090df9f0074012000a4b79f0086027800dd
:101670008502e900050033008b05d1000a85d300ff
:101680008984d3000884d300f9ff3700089fbe0087
:101690000a97be00afb397000700e90021fc2f00b6
:1016a0008f804000008240003fb197008202e90035
:1016b00012003700afb397008703e900a7b79f0078
:1016c00000806200cfb09700615278003e00be00fb
:1016d0002e01be00860378008703e9000500330071
:1016e0008381d1000281d3008180d3000080d300a8
:1016f000f9ff3700009fbe000297be003e00be000b
:101700002e01be00e00f5000e08f5800e00f59009e
:10171000e08f5900d6003400afb397000700e00017
:10172000e4ff3c00d2003700ae60900080c6b300fa
:1017300080cf50000b00320006003c000104e000a6
:10174000080032006640500080cf500073003a001d
:1017500004003700c0c6b30080cf50006f003a00cd
:1017600031003700080178000800e00005003a0069
:101770005e08900081012000a1b79f000000e000fa
:1017800009003200bfb19700110009000381d800a1
:101790008000fd004fb297006440780090df9f000a
:1017a00075012000a5b79f00bfb397001100090085
:1017b0000781d80080017800afb097000100e900f0
:1017c00022fc2f000f014100000241000c003700f5
:1017d000bfb29700110009008501d8000001780010
:1017e000afb397008703e900a7b79f000590b90042
:1017f00000805100cfb097006152780082017800dc
:101800000300e000030034002fb197000200e00065
:10181000efff3c0003007800cf80de00010178007c
:10182000820178003a0037000806be00e00f54003d
:10183000e08f5c0005003a005e0890008301200004
:10184000a3b79f000000e000090032003fb29700fc
:101850006121b9000c00be0086060700cfb29700d8
:101860006540780090df9f0077012000a7b79f00b8
:101870003fb297006121b9000c00be004e06070080
:101880000006be00afb297000500e90027fc2f005c
:101890008f8343008083430097b79f001100370078
:1018a0003fb197006114b9000801be000c00be00f2
:1018b000730607000005be00afb197008301e90081
:1018c000a3b79f000801be002505070000005600d1
:1018d0001fb29700cfb297006552780094b79f006f
:1018e0000a06be00e00f5600e08f5e0003003400e1
:1018f000afb397000700e000e9ff3c004feade00cd
:10190000cfa2de000c00be00040178008401780044
:10191000009fbe000297be0055003700e00f540044
:10192000e08f5c00e00f5d00e08f5d0005003a0095
:101930005e08900081012000a1b79f000000e00038
:101940000d0032003fb1970002027800cfa2de0006
:1019500005037800860378000800be000a01be0077
:10196000d70607004fb297006440780090df9f00d1
:1019700075012000a5b79f003fb1970002027800d3
:10198000cfa2de0005037800860378000800be00c1
:101990000a01be00c3060700009fbe000297be00fa
:1019a000afb197000300e90024fc2f000f024200b2
:1019b0000006420020003700bfb2970005047800ff
:1019c000cfc4de00090578008a0578000802be0051
:1019d0000a03be005fa89700efa897007fa99700b1
:1019e0008fb19700ba060700d0b79f00e1b79f00fc
:1019f000f2b79f0083bf9f00afb397008703e90052
:101a0000a7b79f000802be000a03be003607070002
:101a10005faa970000005200cfb297006556780089
:101a20005fb09700efb097007fb197008fb9970034
:101a3000009fbe000297be003e00be002e01be0009
:101a4000d0af9f00e1af9f00f2af9f0083b79f0030
:101a5000e00f5000e08f5800e00f5900e08f590070
:101a600003003400afb097000100e000d2ff3c005b
:101a70003fb19700e80f510013003a000e1090009c
:101a80000038a30010003200afb19700f78f51006b
:101a900006003e0024fc2f000f024200830042009b
:101aa00000c3b300914f100007003200afb297009f
:101ab0008502e900a5b79f0000c3b30027fc2f00f3
:101ac0008f83430080f37a00afb1970078811100d3
:101ad000120f98006e00900024fc2f000f024200ad
:101ae0008300420081fb07001e0990005e08900001
:101af000800f510006003d0002005000000f9800ca
:101b00000e1090000040a100001798000f00370051
:101b10000000e0000d003d000e1090007400600019
:101b2000f00f500009003a007e089000fe0090007f
:101b3000010050008e08900001005000020050008b
:101b40004240a90001003400000f98004f077800c0
:101b50004f06be004f05be004f04be002f03b1006c
:101b60000000060080007800010037000000e80057
:101b70001004e000fdff3a000100500000000600e4
:101b80008f04b000889fbe008a9fbe008c9fbe005d
:101b90008e1f7800f0b79f0081f79f005001be00b4
:101ba0004000be00f0979f00819f9f00929f9f0082
:101bb000a39f9f0010c6b3000ff19700804f510004
:101bc0001600320010c4b300804f510013003200e1
:101bd000ffb19700530890000000e00003003d00b3
:101be00060002000d00998000c0037000000e000e1
:101bf0000a003a0070c6b3000ff29700804f5200ff
:101c00000300320070c4b300804f520003003a005a
:101c100010002000ffb29700d00a9800ffb0970094
:101c2000c0fa2f000f004000fe010700800178007d
:101c3000e20f500015003a0030002000ffb097007e
:101c40009008980010c6b3000ff19700804f510024
:101c50000a00320064404000804f5100070032000b
:101c60000040e800804f51000400320061ad2000c8
:101c70000040e800804f510001003a00a1ad200073
:101c8000ffb1970063009000160037000000e000ed
:101c900018003400300020007fb29700100a98002e
:101ca00010c6b3008ff2970080cf52000a003200b6
:101cb0006440400080cf5200070032000040e8003e
:101cc00080cf520004003200e1ad20000040e80067
:101cd00080cf520001003a0021ae20007fb1970072
:101ce000620090003158780031587800114878002f
:101cf000c601370014c6b3008ff2970084cf52009c
:101d00000300320010c4b30080cf520013003a0029
:101d10007fb09700600190008200780000c3b3009c
:101d200080587800ffb29700e102980080c7b300a6
:101d30008ff2970084cf52000100320080c5b300bb
:101d4000804878000280e800ffb09700e00098002b
:101d5000710090000080e800f00098000300e000af
:101d600005003a00e3979f0064fb2f000f0142003b
:101d700003077800a001370065ae2000e5b79f009b
:101d800010c6b3008ff0970080cf500005003200de
:101d900010c4b30080cf5000a7003a0072af2000fb
:101da000e2b79f00ffb19700530890001e02200089
:101db0000000e000010035000007e8000e02e80026
:101dc000d4b79f006022b8006033b8007f909700be
:101dd0008f9897001f999700af999700700607009a
:101de000ffb097003102be002103be000000e000fa
:101df00004003d000400be000601be0003f0a20086
:101e0000020037000400be000601be00f0979f00ec
:101e1000819f9f00929f9f00a39f9f006f919700bb
:101e200064015100e2979f00c3fa2f008f814100a7
:101e30006a8041000048eb006b824100c4b79f00fc
:101e400031003700c201200003002000e5fa2f0016
:101e50000f8042009f0107007f9497008f9c97009e
:101e60001f9d9700af9d97000800be000a01be00ad
:101e7000500607000006be005fb1970067015100e1
:101e8000d2b79f004240a9000a003400750607003f
:101e90000002be000203be000800be000a01be0030
:101ea00073060700f0979f00819f9f00929f9f00fd
:101eb000a39f9f00cfb19700678041007100200071
:101ec000050037006f6066004c6add004466de0086
:101ed0000c067200c4eede00e00f5600e08f5e00dc
:101ee000050034008100e900e18f4000f5ff3a0071
:101ef000010037000060eb008100e900fdff3b00be
:101f000067004000c0b79f00dfb297000500e00007
:101f1000090034006022b8006033b8007f90970059
:101f20008f9897001f999700af9997005206070066
:101f30000000e000c3ff3c0060fb2f008f0040006a
:101f40004fb19700010051000000e9008e0f5000d2
:101f500001003d00000778000e00e00003003d0096
:101f600073fb2f000f8141002c003700800f5700ba
:101f700005003d000e80400010409000f3c0b3000b
:101f8000e74f500001003c008041eb00c4fa2f00f5
:101f90000f0242000e0042006a0040008e007800ee
:101fa000010037000000e9008100e90010417800dd
:101fb000834f5100fbff32000107e800efcf5100d3
:101fc00001003a000248e8000100e000030035008b
:101fd00075fb2f000f814200060037000e07e80056
:101fe0006f90970064004000e0979f0061fb2f0016
:101ff0000f8140008e0041008e0178000300370001
:102000001100fb006fb29700e44878008301e900fb
:102010008100e9000300e000f9ff3d00ffb29700f6
:10202000550890000000e000f3003d000e00e900bc
:10203000d00a9800f00037007f9497008f9c97009b
:102040001f9d9700af9d97006022b8006033b800d5
:102050000800be000a01be00d10507000000e00034
:1020600005003d000bf0a200f8979f00899f9f009c
:102070009a9f9f00ab9f9f006f9097007259270017
:102080000280b900026a2800130020007c040700c7
:10209000e4005000e1979f0015003b00e380100032
:1020a000c0ff2f00008460000800ea00e0979f0056
:1020b0007f9097008f9897001f999700af9997008e
:1020c000e9a82000070037000808a3000300320039
:1020d0003902be002903be00ec0507000884d100c8
:1020e000e88444000800e000f7ff3c001b003700d4
:1020f0000100e0001d003400c0ff2f0000806000e0
:10210000e0979f00000478006000b8000200200003
:1021100003ff2300e9a82000070037000808a300f8
:10212000030032003902be002903be00d7050700b4
:102130000884d100e88444000800e000f7ff3c0078
:102140000002be000203be007f9097008f989700a8
:102150001f999700af99970041060700f0979f00dd
:10216000819f9f00929f9f00a39f9f00ffb09700b9
:102170005109900060c6b3008ff1970080cf5100e5
:10218000040032006100200060c4b30080cf510021
:1021900002003a006f929700ea00420001074100f6
:1021a000f30f5700010034003e01200000c3b300cc
:1021b000e0779f0075fb2f008f824200b5b79f002c
:1021c000330037000800be000a01be007905070091
:1021d0000006be00680757004240a9000e00340008
:1021e000a00507000002be000203be000800be00fa
:1021f0000a01be009e0507006022b80046782d0047
:1022000077192400a1050700f0979f00819f9f0088
:10221000929f9f00a39f9f003fb0970068044000db
:10222000890020000d003700a400200005002000d8
:102230000c01be00e0fd2f000f0040002001070050
:102240007fa897008fb097001fb19700afb197009c
:1022500004c3b300046441000006be00e00f560052
:10226000e08f5e00060034008904e900e18f44003d
:10227000edff3a000200370000c3b30000647800ad
:102280008904e900fcff3b0068044400b8b79f00e4
:102290000e00e0000b0034007f9497008f9c9700a5
:1022a0001f9d9700af9d97006022b8006033b80073
:1022b0000800be000a01be006f0507000000e00034
:1022c000c0ff3c00c5fa2f008f8242006a804200a6
:1022d000bfb09700008050008001e9006f91970027
:1022e000e70041006b81420000c3b30001003700ea
:1022f0000201e800924f1000fdff320074fb2f0036
:102300000f00420080804000828050000080410029
:1023100002025000e1979f00ffb29700d50990009c
:1023200060c6b3008ff2970080cf520003003200e6
:1023300060c4b30080cf520002003a008100e80080
:102340000a00370050c6b3008ff0970080cf5000ce
:10235000050032008000eb0050c4b3008ff29700fc
:1023600080cf520001003a00110020000187410097
:102370008e0f520001003d00040778000e00e000bf
:102380001d003500840f570005003d00e2407f002e
:1023900095c3b30040c3b30080cf500001003c00a0
:1023a00005c3b3000e0041008000e9008e017800f3
:1023b000010037008100e9008301e9001142780043
:1023c000854f5200fbff32000307e80090c3b300c3
:1023d00080cf520001003a008448e8000300e0008a
:1023e00005003d000201e9000e07e8006f9097002c
:1023f0000000e800e0979f006f9297008e01780040
:102400008ff097007fb09700ca0007004f07780051
:102410004f06be004f05be004f04be008f04b10042
:1024200000000600889fbe0080047800668440009b
:1024300000ff2700180060004401de00f07f20004c
:10244000800f51000e003a00800ceb001804780059
:102450006f0064001c003a00210090000000e000c2
:1024600019003a00110090000000e00016003a0048
:10247000100020001100e0001400320012003700ac
:102480000200e00005003c0001007800dd010700cb
:10249000000178000000e00008003c00f000280087
:1024a0001800600001fe2300010c700020c02f0006
:1024b000800c41000080eb0004003700800ceb0032
:1024c0000000eb0001003700200020004f04be0098
:1024d00000000600889fbe008a1f78008c9fbe0007
:1024e000000478000206be00e604400019017800ee
:1024f0000200d0004505de008a007800f07f200051
:10250000800f55000c003a006f00610067003a0030
:10251000280090000000e00064003a0018009000dd
:102520000000e00061003a00100020001800e00008
:102530005f0032005d0037000a00e00007003a004b
:1025400008007800af010700800078000000e0007c
:10255000020034000a007800550037006108b90015
:102560000c0140008d814800e07f2000800f510069
:10257000e08f59000d0034001900e00004003d0018
:102580006000b8000200200003ff2f0003003700a6
:102590006000b8000200200003ff2700009cbe007e
:1025a0000294be001000200041003700e00f5100ef
:1025b000e08f590005003400f00028001900600089
:1025c000c410dd00810c700036003700190078005f
:1025d00001002800010360006f0060000040a000bf
:1025e000800c780061015100e0815900c0fc2f008f
:1025f000f1ff2f00800f5100818f590006003d0030
:10260000860c78000000eb0020049800100498006d
:10261000000c780026003700020078000881e800ee
:10262000e400440005003700120c7800110978001e
:1026300099087800800ceb0070004000f00f40001b
:10264000f9ff34008002ea00150032008881e800ba
:1026500070821200980078008508de001300780070
:102660000400dd00008c70006401440093007800d9
:102670008508de00120078000400dd00808970000b
:10268000920078008508de00190078000400dd0063
:1026900000897000190078000500de00800c7800c9
:1026a000990c73000080eb0001003700200020002f
:1026b0004f06be004f0578004f04be000000060024
:1026c0000400fa00889fbe008a9fbe008c1f78001d
:1026d0000006780092bf9f00a3bf9f000404be00c5
:1026e0000401be001fb89700afb89700e4020700ce
:1026f0000005be000001be000800be0098010700f2
:102700001fb99700afb997000000510081805900b0
:1027100020069800310698000a8ebe000c00780052
:102720004f0678004f05be004f04be000080fa003f
:10273000000006000e00fa00889fbe008a9fbe00bf
:102740008c9fbe00000478000145780002067800e6
:1027500083047800840678000300e00002003c0057
:1027600019002000acb4200060c6b300804f5500b3
:102770000e00320060c4b300804f55000b003200e1
:1027800070c6b300804f55000300320070c4b30020
:10279000804f55009c003a00e48f460080003500d1
:1027a00058089000808f56007d003d008d05e800a0
:1027b00060c6b300804f55001000320060c4b30003
:1027c000804f55000d003200081090000038a30023
:1027d00004003a0058089000808f540001003d002a
:1027e000590c9800580890000b005000500c9800ad
:1027f00002003b000000eb00500c98000b00e000d2
:1028000027003c00180990006800900001c3b30045
:10281000017079008201e800130c980058089000bc
:102820000000e00003003c00081090000038a30006
:102830000500320068009000e1c2b30001f07900a9
:102840000280e800100c9800d80890000b00ea0005
:10285000808f500001003d008105ea000b00ea0076
:10286000200c980001804500500c9800890f500002
:1028700001003d0080047800390c98006800900049
:102880009808900001004000090178008c00780051
:1028900016f8070058089000090050001a00370089
:1028a00098089000680090008b8f540018003d003d
:1028b00001004000090178008c0078000bf8070047
:1028c0001808900000814400120c980009805500ff
:1028d000200c9800580890000000e00003003c0025
:1028e000081090000038a30006003200e8009000b5
:1028f000e0c2b30080707900380890000000e80062
:10290000300c980058089000400c9800a600370042
:10291000010040000b0178008c007800f3f70700fd
:102920001808900000814500120c98008b84540018
:10293000580890000000e00003003c0008109000e0
:102940000038a3000500320068009000e1c2b30027
:10295000017079000200e800100c980058089000ff
:10296000890f500001003d0080047800680090004d
:1029700098089000010040008b0046000901780093
:10298000daf707001808900000804400100c980047
:102990005808900009005000200c98008200370071
:1029a00070c6b300804f55000300320070c4b300fe
:1029b000804f550014003a0058089000808f540052
:1029c00004003d00081090000038a30001003a0008
:1029d000590c9800580890000000e900500c98002d
:1029e00002003b000000eb00500c980070c6b300e2
:1029f000804f550002003a005ac6b3000b00370062
:102a00005ac4b3000900370010c6b300804f550008
:102a100002003a000ac7b3000400370010c4b30034
:102a2000804f550001003a000ac5b3001809900014
:102a3000680090003c7079008201e800130c980057
:102a40000c027800580890000000e00003003c00f1
:102a5000081090000038a30017003200e800900032
:102a6000e0c2b30080f079008280e800110c980089
:102a7000580890000000e0000f0034008904e900cd
:102a8000890f500001003d0080047800680090002c
:102a900000804000090178008400780093f7070067
:102aa0001808900000804400100c9800580890000e
:102ab00009005000200c98006800900098089000d1
:102ac000010040000086e8000a5878008000780085
:102ad0000d00e00004003500b0c2b300804878006b
:102ae0008c04780004003700d0c2b300804878001e
:102af0008c0478008d06ea008005eb000a003700a0
:102b0000a20020008d007800708057008900070027
:102b10000fb897009fb897007a81550001f17f00a8
:102b20008b05e800800678000d00e000f4ff3c0013
:102b3000e18f550009003c0050c6b300804f55009e
:102b40000300320050c4b300804f550003003a0028
:102b500000c3b300005e78008c0478000b00e00036
:102b6000040032000b00e900fa80570000804000aa
:102b70000600370000c3b300805c78000500370012
:102b80008b05e90002c3b300a05c41000b00e0002c
:102b9000fbff3c0068009000980890000100400096
:102ba00000805400300c9800081090007400600001
:102bb000f00f50000e003a00780090009808900046
:102bc00001004000a808900001004000b8089000f3
:102bd00001004000c8089000810040007808900083
:102be000808f500002003d0001005000000c980052
:102bf0004f06be004f05be004f04be000080fa0025
:102c00000000060000017800e60140001300780093
:102c100001002800810360006f00600080097800d7
:102c200012003a00220090000000e0000f003a007d
:102c3000120090000000e0000c003a001600200096
:102c40001200e0003800320008003700e4004100c4
:102c5000910978000280e800900878001208780056
:102c60000009eb007003530001003700160020003c
:102c70001300e000f5ff3200e40241000282e800a8
:102c80001100370080004000150078004f00de0082
:102c900080897000950078008180400014007800e1
:102ca0004f00de00808a7000940078008180400030
:102cb000120078004f00de00008a700012007800d9
:102cc000000940000603e90013007800ef0f5000f0
:102cd000ecff36008282e800640241000e003700fb
:102ce0009200d100150078004f00dd0000897000cf
:102cf0009500d100140078004f00dd00808a70003c
:102d00009400d100130078004f00dd00008a7000ad
:102d10009309d1000603e80013007800ff0f50006c
:102d2000efff3e00ef096000938973000600780012
:102d30000000060002027800809fbe00110009001a
:102d40008200d800000178004f00be0002a2b90046
:102d500084805000110098000208780000000600ee
:102d6000020ab900001bb9000200b800810042004d
:102d70008100430000000600889fbe008a9fbe00bd
:102d8000010578000100e0000400350008003c0067
:102d90000000e00020003200050037006000100055
:102da000e080180002003b0001f02c001a00370000
:102db0000004be006011b8006b0920000982cf003a
:102dc000020039000882cf000441b000694252007d
:102dd0000e00320008003b00828171006101640036
:102de0008904d1000884d3008b05e8000442e80080
:102df000f9ff3a00050037000804440089844c00bc
:102e00008b05e9000442e900fbff3a009700070048
:102e10000af0a70001f0a0004f05be004f04be005d
:102e20000000060003f0a200889fbe008a9fbe003b
:102e30008c1f7800b3000700ba0033006450e10033
:102e40004f0032006420e1005200320003826c0027
:102e500007003b000905d0000306d000820f540094
:102e60000c065d0002003900020032008901780082
:102e7000030678008582550004003d000003fd0034
:102e80008103fd008502ea008b854200840f7200f9
:102e900002003b0060001000e08018006011b800e4
:102ea0000005eb007a28e1000a00390006007800ee
:102eb000c75ddd00f707b200878075002d00370081
:102ec000828171000a017800610560008180d10073
:102ed0000080d3008502e900f9ff3b0006044000b2
:102ee0008784480002003b0060041400e0841c005a
:102ef0000988a300070032008a8171008281710075
:102f0000610164008904d1000884d3008b05e800c6
:102f1000170037000978a30013003a000b00e00007
:102f2000130034008b05e9000804440089844c0038
:102f30000a4474000978a3000d003a000b00e00079
:102f4000070034008b05e9000804440089844c0024
:102f500001003a000b0020000978a300f7ff3200bf
:102f60000001eb0002003700828171000a01780045
:102f70003e0007000cf0a70001f0a000720037002f
:102f80006420e10002003a00838f6c00720033007d
:102f90000801be000200be006b003700889fbe0023
:102fa0008a9fbe008c1f7800560007005d0033002a
:102fb00003866c006450e100240032006420e100cc
:102fc000270032006150e100220032006120e10060
:102fd000210032008b854200eb07b1000134b800bc
:102fe000003ab8000804420089844a00013ab80057
:102ff0000030b8008880400009014a000400330016
:103000000000400081804800020149008b05e90072
:10301000c909dd00830170000100320013002000a7
:10302000c814de004814dd004709de001200b200bb
:10303000c808de00088470000c00070001f0a10041
:103040000cf0a70001f0a0003f0037006120e10074
:10305000410032000801be000200be00f7ff370049
:103060006150e100fcff3a003b0037008100200086
:10307000618055000b003d000b00200061fe2f0019
:103080000100e1001d0034008281710061016400d3
:103090008904d1000884d3000000e800faff3a0058
:1030a00071002000610064000300700002006000f5
:1030b0000900320061044400e0844c000988a50046
:1030c000050032008b05e8006808e10002003a00c4
:1030d0008904d1000884d300f20f20000258e100d7
:1030e00005003d00c75ddd00f907b200898075006d
:1030f00008007800000006000bf827008b0078001d
:10310000000005000004be00160007000003be001a
:103110000405be000200be0012000700844f7500c7
:10312000000006000200be006450e1000500360009
:103130006420e100020036000968a30001003a00a3
:103140000800be000160a0004f0678004f05be00d9
:103150004f04be0000000600f0ff2f00f1ff270023
:10316000f9ff3700c70ade00f107b200f50fb20021
:1031700008003200e1cf4200020032000170a000de
:1031800024000500810f70000100320004080500d2
:1031900044000500810f700002003a001400050091
:1031a0008502e9000000400081c04800fcff3b00b0
:1031b0000170a000240005006022b8000602200073
:1031c0000000d0008180d2000482d2008582d2002b
:1031d0000000a0000202520083825a000300310066
:1031e0000202420083824a000000a1000603e900b7
:1031f000f3ff3a000000060081037800d9ff0700c2
:103200000001be006000b8000478a30013003a007b
:103210006220e10015003e000d0039008301d1005d
:103220000281d3008180d3008301d1000281d300c9
:103230008180d3008301d1000281d3008180d3003b
:103240000538b000c42add00f300b20083817200ab
:1032500007f0a70003f0a00000000600f3ff27001e
:10326000f2ff2f006110b900fbff370003ff2700ba
:10327000f7ff3700d0ff07000400be000000060083
:10328000839f68000100e00002003d006000100024
:10329000e08018000300e00002003d006001110022
:1032a000e0811900c4ff07004f00e00002003b006e
:1032b00060001000e080180000000600881f780001
:1032c000000478005001be004000be000400400031
:1032d000858048000601490087814900009cbe00a6
:1032e0000294be000400e1000588e1000690e100c0
:1032f0000798e10002003100680044001008e8006f
:103300004f04780000000600f4874700889fbe0045
:103310008a9fbe008c9fbe008e1f78000205be00f3
:103320000004be00d4b79f00e5b79f00f6b79f002a
:1033300087bf9f000000eb00c0b79f00b0b79f00a1
:10334000a0b79f0090b79f0080b79f000d0420009a
:10335000bfb097004fb09700000140000000e000b0
:103360000f003d004f08de0000007100c0b79f0055
:103370009e00070001003d0012002000a100070090
:1033800001003d0012002000a6000700b100070068
:10339000b60007000f004000c8ff070022003700fa
:1033a0004f08de0000067100ccb79f008f000700b9
:1033b00001003d00120020009200070001003d00c6
:1033c0001200200097000700a20007000fb297002c
:1033d0009fb297002fb39700bfb39700a9000700d3
:1033e0000000520081805a0002015b0083815b0073
:1033f00080b79f0091b79f00a2b79f00b3b79f000f
:103400000007eb009f0007000020e10001a8e10099
:1034100002b0e10003b8e100010031001e0020000d
:103420000e005600c0b79f004fb297000400e000a6
:103430000700350010002000010020006011b800d6
:1034400008047000898470000a0571008b85710082
:103450008d06e900beff3a000400e00003003d00d5
:10346000820007000f00400094ff07004fa897005c
:103470000000e00004003a000fb497009fb49700ea
:103480002fb59700bfb59700940007004f0778004d
:103490004f06be004f05be004f04be004f01b100f5
:1034a00000000600881f780018002000881f7800a0
:1034b00095ff07008f87e9004f04780000000600a1
:1034c000801feb0090ff07008f87e90000000600d7
:1034d000889fbe008a9fbe008c1f78006e00070088
:1034e00007003d0073000700e00f5b00e08f5b000a
:1034f00007003d00320007000006eb000400370023
:103500003400070002003d002a0007001c002000d4
:1035100072000700e3ff07000203be000002be00c6
:103520000c00e00001003200220007000400be0091
:103530000601be004f0678004f05be004f04be00d6
:1035400000000600889fbe008a9fbe008c1f780086
:103550005100070005003d0056000700e00f5b002a
:10356000e08f5b0006003d000400370019000700f3
:1035700003003d006000b8006011b80010000700b3
:1035800056000700ceff07000203be000002be0087
:103590000c00e00001003200060007000400be003d
:1035a0000601be004f0678004f05be004f04be0066
:1035b000000006006000b8006011b800000037008d
:1035c0000402500085825800060359008783590081
:1035d000000006000006eb00e00f5200e08f5a00ea
:1035e000e00f5b00e08f5b00000006000180400000
:1035f00090b79f000001eb008fb097000100e00042
:10360000000006000200700090b79f00018040009b
:1036100080b79f000001eb00ffa897000100e000c9
:10362000000006000200700080b79f00018040008b
:103630006faa9700cf20de0001007000f0af9f005e
:1036400004024200250007004f18de00000272004d
:1036500000000600e4af9f000804440089844c0089
:103660000a054d008b854d00000006003fb2970013
:10367000cfb297005fb39700efb3970000fe2f0023
:10368000000006003fb09700cfb097005fb19700f1
:10369000efb19700000006000205be000004be0066
:1036a000e00f5000e08f5800e00f5900e08f590004
:1036b000000006006000b8006011b8000804500067
:1036c000898458000a0559008b8559001c00200088
:1036d000e00f5200e08f5a00000006000800be0014
:1036e0000a01be0000000600889fbe008a9fbe003f
:1036f0008c1f78000205be000004be000006eb002f
:10370000e00f5000e08f5800e00f5900e08f5900a3
:1037100007003d006000b8006011b80008045000c8
:10372000898458000a0559008b8559001c00200027
:10373000e00f5200e08f5a00e00f5b00e08f5b006b
:1037400002003d000f0007000c00a2000800be00b0
:103750000a01be001c0107000203be000002be00f9
:103760000c00e00001003200060007000400be006b
:103770000601be004f0678004f05be004f04be0094
:10378000000006006000b8006011b800040250009c
:1037900085825800060359008783590000000600ff
:1037a0008f1fd1002a0107008f87e9000000e00089
:1037b000000006001400fa00889fbe008a9fbe0029
:1037c0008c9fbe000004be000205be0068004700da
:1037d0000a90be000890be00460107000070a700d6
:1037e0000bf0a100304320009e0290008082520026
:1037f000b0fe2f000028e10011003d00b0fc2f00ba
:103800000028e100150034001e0990008e08900089
:103810007e0090000501b0000201d1008180d3003c
:103820000080d3008502e800fbff3a000b00e000b7
:103830006b013b0060001000e08018006801370059
:10384000f0ff2f00f1ff27000b00e00064013b00b8
:103850000100280000002000610137006000b8006e
:103860005f0137004f89de00820178006101370077
:1038700007f0a20096013700809feb00f4000700dc
:103880008f87e9000000e000000006002800fa0031
:10389000889fbe008a9fbe008c9fbe0003866b007f
:1038a0003b0107000028a30064003a000128a300a0
:1038b00067003a000008a30062003a000108a30074
:1038c00065003a001e009000be089000810640008e
:1038d000ed3fb100f4805700ee019000111ab800de
:1038e0008e099000311bb8009e099000311cb80071
:1038f000511db800f485570046000700fe019000f6
:103900003a0007008b85e8003e0007008e09900012
:1039100040000700ee019000340007008b85e800ae
:10392000380007008e099000400007009e099000b3
:103930001b18b800890440000a854800fe01900069
:10394000340007008b85e80038000700ee01900086
:10395000300007008e0990001b18b8008904400051
:103960000a8548000a98a30008003a0004024200b1
:1039700085824a0006034b0087834b0008044c00f5
:1039800089844c000a054d008d06e900848272008e
:10399000850273004c3add0085027200010032009e
:1039a00015002000443ade001400b2004538de0065
:1039b000cb45dd000b007000c540de00cb4ddd00c7
:1039c0008b8070004549de00cb55dd000b01710096
:1039d000c551de000d037800ba01070003f0a10015
:1039e0000cf0a70003f0a000fd0037001b18b80082
:1039f0008502400006834800e0834b0060044c00d1
:103a0000070037001b18b8000603400087834800f2
:103a1000faff37001b18b8008703400008844800ed
:103a2000e0844c0060054d00000006001b18b80043
:103a30000804400089844800faff37000108a30009
:103a4000e4003a005800be005801be00e3ff370012
:103a50000008a300df003a0009047800f9ff3700ee
:103a60002800fa00889fbe008a9fbe008c9fbe007f
:103a700003866b00c60007006400e10044003200ca
:103a80006408e1004a0032006100e10046003200b3
:103a90006108e10049003200ec0647006000b80010
:103aa0003d02be003d03be00f48657006011b80021
:103ab0003d04be003d05be007d0320000b00370025
:103ac0000000a0008d06e90013003200040242004d
:103ad00085824a0006034b0087834b0000004000ac
:103ae0008180480002014900838149000802520098
:103af00089825a000a035b008b835b00f0ff3b0066
:103b00000802420089824a000a034b008b834b0063
:103b10008d06e900edff3a00848272008682720011
:103b2000f707b20087827200010032001500200002
:103b30001e0490003e0b900006035400e63fb000c8
:103b40000368a300070032000000a7000500a000e2
:103b50008301d1000281d3008180d3000080d30093
:103b60000603e8008301d1000281d3008180d300e5
:103b70000080d3000002eb000482d2005101070054
:103b800003f0a1000cf0a70003f0a00094003700a0
:103b9000640247006408e1008e0032003400be0079
:103ba0003401be00f6ff37006108e10089003200f1
:103bb0006011b8006000b800f1ff370003ff270074
:103bc00002002000fbff3700889fbe008a9fbe00d6
:103bd0008c9fbe000404b8000506b80089044600a6
:103be00060854e000606b8000a054600e0854e00d6
:103bf0000706b8008b054600040eb800890446008d
:103c00000a854e00e0854d00050eb8000a05460005
:103c10008b854e00060eb8008b0546000416b800d2
:103c20000a0546008b854e000516b8008b05460038
:103c3000041eb8008b0546000800be000a01be0045
:103c40004f06be004f05be004f04be000000060038
:103c5000889fbe008a9fbe008c9fbe000404be00e9
:103c60000605be00809fbe00829fbe004101070086
:103c7000040678000800be000a01be003d010700ee
:103c8000840678004f03be004f02be008d4f7600c1
:103c90007fb0970013003300f0ff2f008b8f6b0075
:103ca00006003b000d0666000c00a7000a00370066
:103cb00007f0a600100020000a003700880f52000d
:103cc000898f5a008a0f5b008b8f5b0003003900dd
:103cd0001000200001003e000000200007f0a700b7
:103ce0000000ea004f06be004f05be004f04be00b4
:103cf00000000600800078005002be005003be00a5
:103d00004439de00f700b200f37f200003016100b8
:103d1000090032000218e10016003a008501720025
:103d200083017300838173000008200015003a00ae
:103d300040002000130037008501720083017300ea
:103d40008381730005003a0004a8be0006a8be00e7
:103d5000100020000b0037000201e90004024200bd
:103d600085824a0006034b0087834b000748a30067
:103d7000f9ff32000740a00004a8be0006a8be005c
:103d800020002000800098009200980000000600ab
:103d9000680447000294be000094be00fc04470083
:103da0008694be008494be0009007800d1ff07000d
:103db00008007800cfff070099007800814f70005d
:103dc0000b003b000800be00fc0007004f00b100e4
:103dd00003003700f3ff2700f2ff2f006110b90046
:103de0004f06be004f05be004f04be000080fa0023
:103df00000000600889fbe00830478000300e000f6
:103e00002c00350003003c000082700004027100a9
:103e10002600320036432000c50020008383cf00f7
:103e20000a0039000541b1008283cf000700390044
:103e30000541b1008183cf00040039000541b10084
:103e40008083cf00010039000541b10085c35300d4
:103e50006022b800120032000a003b008482720027
:103e6000610260008301d1000281d3008180d30010
:103e70000080d3000603e8008743e800f7ff3a001c
:103e8000070037000000400081804800020149001f
:103e9000838149000603e9008743e900f9ff3a00fe
:103ea0008800070009f0a70003f0a0004f04be003f
:103eb0000000060060001000e0801800600119009a
:103ec000e0811900d3ff3b00033e2c00f7ff3700d1
:103ed0002800fa00889fbe008a9fbe008c9fbe000b
:103ee00007067800878669000c003b000304780011
:103ef0008704780008f0a10009f0a100840f5000a9
:103f0000858f5800860f5900890f5c00030033002d
:103f10000cf0a20001003a000cf0a1009cff070089
:103f20006400e1005f003200780147006408e100ae
:103f3000610032006c014700748557003200be00fa
:103f40001201be003a04be001a05be001e03900016
:103f5000be0a90008503530006003d000004fd00ea
:103f60008104fd000205fd008305fd008703ea00d2
:103f7000050378000df8a30004003200600414006b
:103f8000e0841c0060051d00e0851d006022b80073
:103f90007d0320000d38e1008006eb000b003900a6
:103fa0004433dd00f300b2008301730039003700b1
:103fb000848272000d027800e10664008b85d100d6
:103fc0000a85d3008984d3000884d3008703e900dd
:103fd000f7ff3b0008004000898048000a014900c3
:103fe0008b81490004003b0060001000e080180055
:103ff00060011900e08119000358a3000900320094
:104000008d82720084827200610260008301d1009f
:104010000281d3008180d3000080d3000603e80032
:104020001b0037000348a30017003a000600e00019
:10403000170034000603e9000d00a300000048004b
:104040008180480002014900838149000348a300a0
:104050000f003a000600e000090034000603e90002
:10406000000040008180480002014900838149002e
:1040700001003a000003eb000348a300f5ff320003
:104080006022b800020037008482720061826600fc
:104090000c00070003f0a1000cf0a70003f0a00043
:1040a0004fff3700640147006408e10002003a0056
:1040b0000df8a30047ff3a003200be001201be0017
:1040c00047ff370018002000570020000804530065
:1040d0000d003d000600200097fc2f000740e10086
:1040e0001e00340084827200610260008301d100ee
:1040f0000281d3008180d3000080d3000804e8004f
:10410000f8ff3a00470020006104600005047400d5
:10411000040464000d00320061004000e0804800ab
:1041200060014900e081490003b8a50007003200a2
:104130000603e8006538e10004003a008301d1007d
:104140000281d3008180d3000080d300f87f20005b
:104150000830e10003003500080378006000b80073
:104160006011b8004433dd00f300b2008301730036
:104170000000060005ff27000582610007003200ed
:104180000428e100010032002400050006000700b9
:1041900001003a0044000500040805000200070081
:1041a000f9ff3a00140005006f826100810270007f
:1041b000850271008502720000000600e482400062
:1041c0001078a30007003200640240001178a300b9
:1041d0003400be001401be00040032000330a7000a
:1041e000000006003500be001501be000330a0002f
:0441f00000000600c5
:020000040000fa
:020000040005f5
:0457f400021e000091
:020000040000fa
:020000040005f5
:0457f800bdfa0000f6
:020000040000fa
:020000040005f5
:0457fc007f3e0000ec
:020000040000fa
:100008002e3b00002e3b00002e3b00002e3b000044
:100018002e3b00002e3b00002e3b00002e3b000034
:100028002e3b00002e3b00002e3b00002e3b000024
:100038002e3b00002e3b00002e3b00008a360000bd
:100048002e3b00002e3b00002e3b0000282d000018
:10005800102d00002e3b00002e3b00002e3b000020
:100068002e3b00002e3b00002e3b00002e3b0000e4
:100078002e3b00002e3b00002e3b00002e3b0000d4
:100088002e3b00002e3b00002e3b00002e3b0000c4
:100098002e3b00002e3b00007e2d0000662d000048
:1000a8002e3b00002e3b00002e3b00002e3b0000a4
:1000b8002e3b00002e3b00002e3b00002e3b000094
:1000c8002e3b00002e3b00002e3b00002e3b000084
:1000d8002e3b00002e3b00002e3b00002e3b000074
:1000e8002e3b00002e3b00002e3b00002e3b000064
:1000f8002e3b00002e3b00002e3b00002e3b000054
:100108002e3b00002e3b00002e3b00002e3b000043
:100118002e3b00002e3b00002e3b00002e3b000033
:100128002e3b00002e3b00002e3b00002e3b000023
:100138002e3b00002e3b00002e3b00002e3b000013
:100148002e3b00002e3b00002e3b00002e3b000003
:100158002e3b00002e3b00002e3b00002e3b0000f3
:100168002e3b00002e3b00002e3b00002e3b0000e3
:100178002e3b00002e3b00002e3b00002e3b0000d3
:100188002e3b00002e3b00002e3b00002e3b0000c3
:100198002e3b00002e3b00002e3b00002e3b0000b3
:1001a8002e3b00002e3b00002e3b00002e3b0000a3
:1001b8002e3b00002e3b00002e3b00002e3b000093
:1001c8002e3b00002e3b00002e3b00002e3b000083
:1001d8002e3b00002e3b00002e3b00002e3b000073
:1001e8002e3b00002e3b00002e3b00002e3b000063
:0801f8002e3b00002e3b00002d
:020000040000fa
:100208002e3b00002e3b00002e3b00002e3b000042
:100218002e3b00002e3b00002e3b00002e3b000032
:100228002e3b00002e3b00002e3b00002e3b000022
:100238002e3b00002e3b00002e3b00008a360000bb
:100248002e3b00002e3b00002e3b0000282d000016
:10025800102d00002e3b00002e3b00002e3b00001e
:100268002e3b00002e3b00002e3b00002e3b0000e2
:100278002e3b00002e3b00002e3b00002e3b0000d2
:100288002e3b00002e3b00002e3b00002e3b0000c2
:100298002e3b00002e3b00007e2d0000662d000046
:1002a8002e3b00002e3b00002e3b00002e3b0000a2
:1002b8002e3b00002e3b00002e3b00002e3b000092
:1002c8002e3b00002e3b00002e3b00002e3b000082
:1002d8002e3b00002e3b00002e3b00002e3b000072
:1002e8002e3b00002e3b00002e3b00002e3b000062
:1002f8002e3b00002e3b00002e3b00002e3b000052
:100308002e3b00002e3b00002e3b00002e3b000041
:100318002e3b00002e3b00002e3b00002e3b000031
:100328002e3b00002e3b00002e3b00002e3b000021
:100338002e3b00002e3b00002e3b00002e3b000011
:100348002e3b00002e3b00002e3b00002e3b000001
:100358002e3b00002e3b00002e3b00002e3b0000f1
:100368002e3b00002e3b00002e3b00002e3b0000e1
:100378002e3b00002e3b00002e3b00002e3b0000d1
:100388002e3b00002e3b00002e3b00002e3b0000c1
:100398002e3b00002e3b00002e3b00002e3b0000b1
:1003a8002e3b00002e3b00002e3b00002e3b0000a1
:1003b8002e3b00002e3b00002e3b00002e3b000091
:1003c8002e3b00002e3b00002e3b00002e3b000081
:1003d8002e3b00002e3b00002e3b00002e3b000071
:1003e8002e3b00002e3b00002e3b00002e3b000061
:0803f8002e3b00002e3b00002b
:020000040000fa
:1041f4004d4500004f5700000d0a0000004200002a
:1042040049540000202500006420000049530000a8
:1042140020480000490d00000a0000004249000047
:1042240054200000256400002049000053200000b1
:104234004c4f00000d0a0000000d00000a61000050
:104244006e6100006c6f000067310000203d0000cb
:1042540020250000660d00000a0000000d0a000081
:10426400616e0000616c00006f6700003220000086
:104274003d200000256600000d0a0000000d00002e
:104284000a6100006e6100006c6f0000673300007b
:10429400203d000020250000660d00000a000000fb
:1042a4000d0a00005265000074750000726e000073
:1042b4006564000020560000616c00007565000014
:1042c400203d000020250000660d00000a000000cb
:1042d400313200003a330000383a00003134000033
:1042e400004f00006374000020200000362000000e
:1042f4003230000031310000000d00000a46000099
:104304004f43000045200000434800004153000093
:1043140053490000532000004c6f00007720000038
:10432400566f00006c740000616700006520000097
:104334004c6f0000616400002053000077690000a6
:10434400746300006865000072200000424f0000a2
:10435400415200004420000042750000696c0000d6
:10436400742000006f6e0000202500007320000000
:104374006174000020250000730d00000a00000095
:1043840020090000004500005252000020250000d2
:1043940030340000640d00000a00000052440000a4
:1043a400590d00000a0000004745000054000000b9
:1043b4005345000054000000434c000045410000f8
:1043c400527c0000434c00005200000048450000ad
:1043d4004c4c00004f2000004b4900005454000096
:1043e4005900000000000000d6a10000bc2d000010
:1043f400daa10000cc2d0000dea10000dc2d0000bd
:10440400e8a10000ec2d0000f4a100000000000071
:10441400444900004e000000444f00005554000081
:104424000041000044430000000000000aa2000014
:10443400fc2d00000ea200003c2e000013a2000080
:10444400b02e0000f4a10000000000000ea2000045
:104454007c2e0000f4a10000000000000ea2000069
:10446400962e0000f4a100000000000000000000ef
:104474000000000000000000000000000000000038
:104484000000000000000000000000000000000028
:104494000000000000000000000000000000000018
:1044a40000000000000000000000000020090000df
:1044b40000200000003000003132000033340000de
:0c44c400353600003738000039000000d9
:020000040000fa
:1044d0000000fa002c03a8002c23a8002c43a800fd
:1044e0002c63a8002c83a8002ca3a8002cc3a80030
:1044f0002ce3a8002d03a8002d23a8002d43a8001d
:104500002d63a8002d83a8002da3a8002dc3a8000b
:104510002de3a800c862a900c8c2a900c8e2a9008a
:10452000c902a900c922a900c942a900c962a900fb
:10453000c982a900c9a2a900c9c2a900c9e2a900eb
:10454000d1a2a900d1c2a900d8e2a900d902a9002c
:10455000d962a900e002a900e022a900e042a90076
:10456000e062a900e082a900e0a2a900e0c2a900df
:10457000e802a900e822a900e842a900e862a9002f
:10458000e882a900e8a2a900e8c2a900f042a900b7
:10459000f062a900d802a800d822a800d842a8003a
:1045a000d862a800d882a800d8a2a800d8c2a800c3
:1045b000e0e2a80000000000e402a9000000000002
:1045c000e422a90000000000e442a900000000006d
:1045d000e462a90000000000e482a80000000000de
:1045e000e4a2a80000000000e4c2a900000000004e
:1045f000dd62a80000000000ec02a800000000003e
:10460000ec22a80000000000ec42a800000000001e
:10461000ec62a80000000000ec82a800000000008e
:10462000eca2a80000000000ecc2a80000000000fe
:10463000f442a80000000000cc62a80000000000c6
:10464000ccc2a80000000000cce2a80000000000de
:10465000cd02a80000000000cd22a800000000004c
:10466000cd42a80000000000cd62a80000000000bc
:10467000cd82a80000000000cda2a800000000002c
:10468000cdc2a80000000000cde2a800000000009c
:10469000f462a80000000000dd02a8000000000095
:1046a000d5a2a80000000000d5c2a80000000000ac
:1046b000dce2a8000080fa00000006000800fa0012
:1046c000000f7800110798001e0090000000e00025
:1046d00002003200100020001007980000000000c7
:1046e0001e0078006101b900220798003307980086
:1046f000f0012000010020002e019000be0190007a
:10470000800f5100818f590075013e002e009000ee
:10471000be009000006001001f0037002800370035
:10472000320037003c0037004600370050003700a9
:104730005a003700640037006e00370077003700fa
:10474000810037008b003700950037009f0037004d
:10475000a9003700b3003700bd003700c70037009d
:10476000d1003700d8003700e1003700eb003700f8
:10477000f5003700ff00370009013700130137004b
:104780001d013700240137002e01370037013700a3
:10479000410137004b0137001e009000614060006e
:1047a00061416000412e200091407800e0cfb300cd
:1047b00000c0600002407000e4e2b700480137002a
:1047c0001e009000614060006140600000414000b8
:1047d000412e200091407800d0cfb30000c060008f
:1047e00002407000e4e2b7003d0137001e00900077
:1047f00061406000614060004201dd00412e200008
:1048000091407800b0cfb30000c06000024070005b
:10481000e4e2b700320137001e0090006140600002
:10482000614060004301dd00412e2000914078008e
:1048300070cfb30000c0600002407000e4e2b70037
:10484000270137001e009000614060006140600059
:104850004401dd00412e200091407800f0ceb300ed
:1048600000c0600002407000e4e2b7001c013700a5
:104870001e00900061406000614060004501dd0065
:10488000412e200091407800f0cdb30000c06000c0
:1048900002407000e4e2b700110137001e009000f2
:1048a00061406000614060004601dd00412e200053
:1048b00091407800f0cbb30000c06000024070006f
:1048c000e4e2b700060137001e009000614060007e
:1048d000614060004301dd00d12d2000914078004f
:1048e00070cfb30000c0600002407000dde2b7008e
:1048f000fb0037001e0090006140600061416000d5
:10490000c12e200091407800e0cfb30000c06000cd
:1049100002407000ece2b700f10037001e0090008a
:10492000614060006140600000414000c12e2000f5
:1049300091407800d0cfb30000c06000024070000a
:10494000ece2b700e60037001e0090006140600016
:10495000614060004201dd00c12e200091407800de
:10496000b0cfb30000c0600002407000ece2b700be
:10497000db0037001e009000614060006140600075
:104980004301dd00c12e20009140780070cfb300bc
:1049900000c0600002407000ece2b700d0003700b9
:1049a0001e00900061406000614060004401dd0035
:1049b000c12e200091407800f0ceb30000c060000e
:1049c00002407000ece2b700c50037001e00900006
:1049d00061406000614060004501dd00c12e2000a3
:1049e00091407800f0cdb30000c06000024070003c
:1049f000ece2b700ba0037001e0090006140600092
:104a0000614060004601dd00c12e20009140780029
:104a1000f0cbb30000c0600002407000ece2b700d1
:104a2000af0037001e0090006140600061406000f0
:104a30004201dd00412f200091407800b0cfb3004b
:104a400000c0600002407000f4e2b700a40037002c
:104a50001e00900061406000614060004301dd0085
:104a6000c12c20009140780070cfb30000c06000de
:104a700002407000cce2b700990037001e009000a1
:104a800061406000614060004601dd00c12c2000f3
:104a900091407800f0cbb30000c06000024070008d
:104aa000cce2b7008e0037001e009000614060002d
:104ab000c700dd00ccc2bf000074a100014070003f
:104ac000cce2b700860037001e0090006140600015
:104ad00061416000d12c200091407800e0cfb3000c
:104ae00000c0600002407000cde2b7007c003700db
:104af0001e00900061406000614060000041400085
:104b0000d12c200091407800d0cfb30000c06000cd
:104b100002407000cde2b700710037001e00900027
:104b200061406000614060004201dd00d12c200046
:104b300091407800b0cfb30000c060000240700028
:104b4000cde2b700660037001e00900061406000b3
:104b5000614060004301dd00d12c200091407800cd
:104b600070cfb30000c0600002407000cde2b7001b
:104b70005b0037001e0090006140600061406000f3
:104b80004401dd00d12c200091407800f0ceb3002c
:104b900000c0600002407000cde2b7005000370056
:104ba0001e00900061406000614060004501dd0032
:104bb000d12c200091407800f0cdb30000c06000ff
:104bc00002407000cde2b700450037001e009000a3
:104bd00061406000614060004601dd00d12c200092
:104be00091407800f0cbb30000c06000024070003c
:104bf000cde2b7003a0037001e009000614060002f
:104c0000c700dd00cdc2bf000074a10001407000ec
:104c1000cde2b700320037001e0090006140600016
:104c2000614060004301dd00412f20009140780089
:104c300070cfb30000c0600002407000f4e2b70023
:104c4000270037001e009000614060006141600055
:104c5000d12d200091407800e0cfb30000c060006b
:104c600002407000dde2b7001d0037001e0090001a
:104c700061406000614060004501dd00512d200071
:104c800091407800f0cdb30000c060000240700099
:104c9000d5e2b700120037001e00900061406000ae
:104ca000614060004601dd00512d200091407800f8
:104cb000f0cbb30000c0600002407000d5e2b70046
:104cc000070037001e00900061406000c700dd0053
:104cd000dcc2bf000074a10001407000dce2b7003c
:104ce0000080fa00000006000800fa00000f7800bb
:104cf000000000000000eb00f05188001e0078006a
:104d00006101b9002207980033079800f0012000e4
:104d1000010020002e019000be019000800f510084
:104d2000818f5900f8003e002e009000be009000d8
:104d3000006001001f003700230037002900370002
:104d40002f003700350037003b00370041003700a7
:104d5000470037004d00370051003700570037003b
:104d60005d00370063003700690037006f003700cf
:104d7000750037007b00370081003700870037005f
:104d80008c00370090003700960037009c003700f9
:104d9000a2003700a8003700ae003700b40037008b
:104da000b9003700bf003700c3003700c900370023
:104db000cf003700e4c2bf00614060000080fb000c
:104dc00010079800d2003700e4c2bf000080fb004b
:104dd0000000d100614060000080fb0010079800d7
:104de000cb003700e4c2bf000080fb004200de00c1
:104df000614060000080fb0010079800c40037008d
:104e0000e4c2bf000080fb004300de0061406000a0
:104e10000080fb0010079800bd003700e4c2bf000f
:104e20000080fb004400de00614060000080fb0069
:104e300010079800b6003700e4c2bf000080fb00f6
:104e40004500de00614060000080fb001007980014
:104e5000af003700e4c2bf000080fb004600de0068
:104e6000614060000080fb0010079800a800370038
:104e7000ddc2bf000080fb004300de006140600037
:104e80000080fb0010079800a1003700ecc2bf00b3
:104e9000614060000080fb00100798009c00370014
:104ea000ecc2bf000080fb000000d1006140600048
:104eb0000080fb001007980095003700ecc2bf008f
:104ec0000080fb004200de00614060000080fb00cb
:104ed000100798008e003700ecc2bf000080fb0076
:104ee0004300de00614060000080fb001007980076
:104ef00087003700ecc2bf000080fb004400de00ea
:104f0000614060000080fb001007980080003700bf
:104f1000ecc2bf000080fb004500de006140600085
:104f20000080fb001007980079003700ecc2bf003a
:104f30000080fb004600de00614060000080fb0056
:104f40001007980072003700f4c2bf000080fb0019
:104f50004200de00614060000080fb001007980006
:104f60006b003700ccc2bf000080fb004300de00b6
:104f7000614060000080fb0010079800640037006b
:104f8000ccc2bf000080fb004600de006140600034
:104f90000080fb00100798005d003700ccc2bf0006
:104fa0000080fb004700de000080fb001007980037
:104fb00057003700cdc2bf00614060000080fb0099
:104fc0001007980052003700cdc2bf000080fb00e0
:104fd0000000d100614060000080fb0010079800d5
:104fe0004b003700cdc2bf000080fb004200de0056
:104ff000614060000080fb0010079800440037000b
:10500000cdc2bf000080fb004300de0061406000b5
:105010000080fb00100798003d003700cdc2bf00a4
:105020000080fb004400de00614060000080fb0067
:105030001007980036003700cdc2bf000080fb008b
:105040004500de00614060000080fb001007980012
:105050002f003700cdc2bf000080fb004600de00fd
:10506000614060000080fb001007980028003700b6
:10507000cdc2bf000080fb004700de000080fb00c7
:105080001007980022003700f4c2bf000080fb0028
:105090004300de00614060000080fb0010079800c4
:1050a0001b003700ddc2bf00614060000080fb00d4
:1050b0001007980016003700d5c2bf000080fb0023
:1050c0004500de00614060000080fb001007980092
:1050d0000f003700d5c2bf000080fb004600de0095
:1050e000614060000080fb00100798000800370056
:1050f000dcc2bf000080fb004700de000080fb0038
:1051000010079800020037008000eb00110798009c
:105110001e0090000080fa00000006000600fa0061
:105120002007980010002000000f78000000eb001e
:10513000100798000b0037002e0090001e00600042
:10514000800078001e0090005cfd07001e007800c3
:1051500000004000000f78001e0090000000e800f2
:10516000100798001e009000ff0f5000f2ff34005f
:105170000080fa00000006000600fa00100020007f
:10518000100798000000eb00000f78000000eb0013
:10519000200798000c0037002e009000d2fe070078
:1051a0000000e000020032001e0090001e0f4000d0
:1051b0001e00900000004000100798002e00900094
:1051c0000000e800200798002e009000ff0f50001c
:1051d000f1ff34001e0078000080fa000000060095
:1051e0000800fa00000f7800000000000000eb004b
:1051f000f05188001e0078006101b9002207980074
:1052000033079800f0002000010020002e019000dc
:10521000be019000800f5100818f590060003e0058
:105220002e009000be009000006001000f003700cb
:1052300013003700190037001f0037002500370022
:105240002b00370031003700370037003c003700b3
:105250003e0037004000370042003700440037006e
:1052600046003700480037004a003700dac2bf0066
:10527000614060000080fb00100798004a00370082
:10528000dac2bf000080fb000000d1006140600076
:105290000080fb001007980043003700dac2bf000f
:1052a0000080fb004200de00614060000080fb00e7
:1052b000100798003c003700dac2bf000080fb00f6
:1052c0004300de00614060000080fb001007980092
:1052d00035003700dac2bf000080fb004400de006a
:1052e000614060000080fb00100798002e0037002e
:1052f000dac2bf000080fb004500de0061406000b4
:105300000080fb001007980027003700dac2bf00ba
:105310000080fb004600de00614060000080fb0072
:105320001007980020003700e2c2bf000080fb0099
:105330004700de000080fb00100798001a003700cd
:10534000f15180001107980017003700f2518000da
:105350001207980014003700f351800013079800db
:1053600011003700f0518000100798000e00370040
:10537000f1518000110798000b003700f2518000b6
:105380001207980008003700f351800013079800b7
:1053900005003700f0518000100798000200370028
:1053a0008000eb00110798001e0090000080fa00ba
:1053b000000006000600fa00100020001007980008
:1053c0000000eb00000f78000000eb0020079800c1
:1053d0000c0037002e00900081ff07000000e00065
:1053e000020032001e0090001e0f40001e009000c0
:1053f00000004000100798002e0090000000e80018
:10540000200798002e009000ef0f5000f1ff3400ad
:105410001e0078000080fa00000006000200fa007a
:105420000000eb00000f7800270037009e01780095
:105430001e0078004700dd008000780040812000d9
:105440000080400000017800c318dd00408020008b
:1054500000804000020878001e0078004300dd0054
:105460008080e80040802000808040000000eb0049
:10547000800878001e0078004300dd00e400400052
:1054800040802000808040000000eb008008780011
:105490001e0078004300dd00e60040004080200050
:1054a00080804000f0072000800878001e0078000f
:1054b0008000400040912000808040000000eb0010
:1054c000800878001e0fe800100020009e0f1000da
:1054d000d6ff3400b00020004011880021e2a8006f
:1054e00020a2a9002062a90000402000101188001d
:1054f0008560a9008580a900910a2000914078006c
:10550000f0c8b30000c0600001c6b30001407000e5
:10551000a9e0b700a10a20009140780080cfb30035
:1055200000c060000014a000aae0b7009560a800c9
:105530009580a900b0002000c011880031e2a800c9
:1055400030a2a9003062a90000402000901188001c
:1055500087c0a90087e0a900310b200091407800a6
:1055600080cfb30000c060006040b300b3e0b7007c
:10557000310b200091407800f0c8b30000c06000fb
:1055800001c2b30001407000b3e0b70097c0a800ab
:1055900097e0a9000080fa00000006000a00fa0067
:1055a00010079800210798001e00900040079800ff
:1055b0004e009000e10f5000090032004e009000b4
:1055c000e20f500006003200ae0090000040eb00f9
:1055d000804878000000eb00300798000d0037008d
:1055e0000a0807001e0090004300dd0080007800dc
:1055f0004080200068005000808040002e00900015
:1056000056070700000f78000a0807001e00780000
:10561000300798003e0090000080fa00000006006d
:105620000c00fa0010079800414798001e009000f7
:10563000400798004e009000e10f50000400320037
:105640004e009000e20f5000080032000e003700bc
:1056500023c2bf000080fb000000d1006140600059
:105660000080fb00000f78000900370033c2bf0044
:105670000080fb000000d100614060000080fb0062
:10568000000f78000200370010002000000f7800a3
:105690001e00e00015003a001e0090005007980020
:1056a0005e009000e10f5000040032005e009000a8
:1056b000e20f5000070032000c0037004e4090000f
:1056c0000080fb00201188001000200030079800a7
:1056d000080037004e4090000080fb00a0118800b9
:1056e0001000200030079800020037000000eb0097
:1056f000300798003e0090000080fa00000006008d
:105700000600fa0010079800210798000000eb003f
:10571000000f78000b0037001e0078008000780032
:105720002e009000008040001040780080407800fb
:105730001e009000baff07000000e00001003200e8
:105740001e0fe8001e007800800078002e009000f8
:1057500000804000104078000004e000eeff3a00b6
:105760000000eb000080fa00000006000800fa00cc
:10577000100798001e009000300798003e0090002f
:10578000e10f5000060032003e009000e20f500092
:10579000030032000000eb00200798000c003700e7
:1057a0009a0707001e0090004300dd00800078008b
:1057b0004080200068005000008040001307070070
:1057c000000f78009b0707001e0078002007980054
:1057d0002e0090000080fa00000006000600fa008b
:1057e000100798001e009000200798002e009000df
:1057f000e10f5000040032002e009000e20f500034
:10580000080032000e00370023c2bf000080fb00fa
:105810000000d100614060000080fb00000f7800b4
:105820000900370033c2bf000080fb000000d10038
:10583000614060000080fb00000f7800020037002c
:1058400010002000000f78001e0078000080fa0091
:10585000000006000600fa00000f78001e00780025
:10586000200798002e009000e10f50000400320045
:105870002e009000e20f5000080032000e003700aa
:105880001e00780080004000409120000080400011
:105890001000780010079800090037001e007800fb
:1058a00080004000409120000080400010007800ff
:1058b00010079800020037000000eb001007980066
:1058c0001e0090000080fa00000006000400fa00ac
:1058d000000f78001e007800100798001e0090004e
:1058e000e10f5000040032001e009000e20f500053
:1058f00001003200060037001e00780080004000e2
:1059000040912000808040000000eb00800878007b
:105910000080fa00000006000800fa001007980056
:105920001e009000200798002e009000e10f50000c
:10593000040032002e009000e20f500001003200ff
:105940001f003700310707001e0090004300dd00f4
:1059500080007800408020006800500000804000f7
:10596000a00607001e009000300798003e0090003f
:10597000e10f5000060032003e009000e20f5000a0
:105980000a0032000d00370030118000000f78004f
:1059900022c2bf00614060000004e000faff3a004c
:1059a00006003700b0118000000f780032c2bf003f
:1059b000614060000004e000faff3a001d070700a4
:1059c0000080fa00000006000400fa00000f7800d2
:1059d0001e007800100798001e009000e10f500094
:1059e000040032001e009000e20f5000060032005a
:1059f000090037002342a900000000002342a8004c
:105a000000000000040037003342a900000000003d
:105a10003342a800000000000080fa0000000600e9
:105a2000809fbe000000fa0000408000114080000e
:105a300061004000e080480000408800114088007c
:105a40008580a9000080fa004f00be0000400600db
:105a5000809fbe000000fa00140037003040800034
:105a60008000e8005040800080806000404080005e
:105a7000808f500003003a0010002000a0488800ea
:105a80000a003700214080003040800080804000c4
:105a90003011800080487800304080008000e800ad
:105aa00050408000008060003040880022c2bf006b
:105ab000614060000004e000e8ff3a008560a90052
:105ac0000080fa004f00be0000400600809fbe002c
:105ad0000000fa000040800011408000610040009a
:105ae000e0804800004088001140880087e0a9005d
:105af0000080fa004f00be0000400600809fbe00fc
:105b00000000fa0014003700704080008000e800b8
:105b1000904080008080600080408000808f500036
:105b200003003a0010002000b04888000a00370047
:105b3000614080007040800080804000b011800093
:105b400080487800704080008000e800904080002d
:105b5000008060007040880032c2bf006140600079
:105b60000004e000e8ff3a0087c0a9000080fa00c6
:105b70004f00be00004006000200fa00000f78004f
:105b80005200200081212a001e0078005a030700dd
:105b90000080fa00000006000200fa00000f780002
:105ba0005200200081222a001e00780052030700c4
:105bb0000080fa00000006000200fa00000f7800e2
:105bc0005200200001232a001e0078004a0307002b
:105bd0000080fa00000006000200fa00000f7800c2
:105be000a10f2a0010002000c5fe07000000eb00f6
:105bf0000080fa00000006000400fa001007980078
:105c0000a20020008000eb001e00900058ea070070
:105c1000000f78001e00780071fd07000000e00012
:105c2000080032001e007800801f780010102a0043
:105c3000801f780080912000e7ea0700e487570082
:105c4000070037001e007800801f780000112a002e
:105c5000801f780080912000dfea0700e48757006a
:105c60008191200010002000a5fe07000000eb003d
:105c70000080fa00000006000400fa0010079800f7
:105c8000a20020008000eb001e00900038ea070010
:105c9000000f78001e00780013fc07000000e000f1
:105ca000080032001e007800801f780010102a00c3
:105cb000801f780080912000c7ea0700e487570022
:105cc000070037001e007800801f780000112a00ae
:105cd000801f780080912000bfea0700e48757000a
:105ce000819120001000200085fe07000000eb00dd
:105cf0000080fa00000006000400fa001007980077
:105d0000a20020008000eb001e00900018ea0700af
:105d1000000f7800110020001e00780067fa0700cd
:105d20000000eb000080fa00000006000400fa000a
:105d300010079800a20020008000eb001e009000d9
:105d40000bea0700000f78008000eb001e007800cf
:105d50005afa07000000eb000080fa00000006007d
:105d60001c00fa00300f9800a20020008000eb0019
:105d70003e089000fee90700200f98000000eb00ad
:105d8000100f98000000eb00000f98000000eb00df
:105d9000700798000000eb00600798000000eb001f
:105da000500798000000eb00400798000000eb004f
:105db000300798000000eb00200798006000b80052
:105dc000008fbe002e089000500f9800de08900053
:105dd000e18f5000110032005e089000e10f50008a
:105de00004003c00de0890000100e00008003200e2
:105df000130037005e089000e20f50000a003200e6
:105e0000de089000e38f50000a0032000c003700db
:105e100070092000200798000a003700700d20004c
:105e20002007980007003700700a2000200798001c
:105e300004003700700e2000200798000100370092
:105e400064003700100020006500070060c2a90050
:105e500030002000e0050700000000002e00900048
:105e6000dd0507000000eb00db050700100f9800c0
:105e70000000eb00d8050700000f98000000eb00c1
:105e8000d505070070079800300620005400070071
:105e90001e089000801f7800f0112a00801f7800f3
:105ea000809520004cea0700e48757008195200088
:105eb0001000200012fe07008e089000811f78005d
:105ec00000132a00801f78008095200042ea070016
:105ed000e4875700819520001000200008fe07008d
:105ee0007e009000801f780010142a00801f780028
:105ef0008095200038ea0700e4875700819520004c
:105f000010002000fefd07009e0890006107980029
:105f10006e0090004800dd00600798008e08900039
:105f2000f00f2000808060006e0090000100700083
:105f3000600798006e009000000040006007980025
:105f40007e0090004700de00700798000000eb0024
:105f5000500798005e0090004800dd005007980050
:105f6000fe009000f00f2000808060005e00900036
:105f70000100700050079800ee0090005e00900055
:105f800000807000400798000001eb00ce009000f8
:105f90002e089000c4000700cf80de0076f30700d3
:105fa000008fbe001e00be00809fbe0020152a008c
:105fb000801f78008095200007ea0700e6875700d9
:105fc0008195200010002000cdfd07000000eb00af
:105fd000400f98004e0890000080fa000000060074
:105fe0000400fa00000f78001e00780010079800e7
:105ff0001e009000e30f50004a0032001e00900087
:10600000e30f50000a003c001e009000e10f50001a
:10601000240032001e009000e10f500031003c00cf
:106020001e0090000000e0000e0032008d003700de
:106030001e009000e50f50005a0032001e00900034
:10604000e50f5000470035001e009000e60f50009d
:10605000640032001e009000e70f50007100320013
:10606000800037008000eb000000eb0093f9070090
:106070008000eb001000200090f907008000eb008a
:10608000200020008df907008000eb003000200088
:106090008af907008000eb004000200087f9070024
:1060a0007f0037008000eb000000eb0083f9070061
:1060b0008000eb001000200080f907008000eb005a
:1060c000200020007df90700110020003000200092
:1060d0007af907008000eb004000200077f9070004
:1060e0006f0037008000eb000000eb0073f9070041
:1060f0008000eb001000200070f907001100200064
:10610000200020006df907008000eb003000200027
:106110006af907008000eb004000200067f90700e3
:106120005f0037008000eb000000eb0063f9070020
:106130008000eb001000200060f907001100200033
:10614000200020005df90700110020003000200031
:106150005af907008000eb004000200057f90700c3
:106160004f0037008000eb000000eb0053f9070000
:10617000110020001000200050f907008000eb0003
:10618000200020004df907008000eb0030002000c7
:106190004af907008000eb004000200047f90700a3
:1061a0003f0037008000eb000000eb0043f90700e0
:1061b000110020001000200040f907008000eb00d3
:1061c000200020003df907001100200030002000d1
:1061d0003af907008000eb004000200037f9070083
:1061e0002f0037008000eb000000eb0033f90700c0
:1061f000110020001000200030f9070011002000dd
:10620000200020002df907008000eb003000200066
:106210002af907008000eb004000200027f9070062
:106220001f0037008000eb000000eb0023f907009f
:10623000110020001000200020f9070011002000ac
:10624000200020001df90700110020003000200070
:106250001af907008000eb004000200017f9070042
:106260000f0037008000eb000000eb0013f907007f
:106270008000eb001000200010f907008000eb0008
:10628000200020000df907008000eb003000200006
:106290000af90700110020004000200007f907005c
:1062a0000080fa00000006005200fa002017980053
:1062b00031179800421798006400470081232a0094
:1062c0000f000900311878000002b1004e11900053
:1062d00072279800fe219000e18f51001b003200d0
:1062e0007e209000e20f50002c003200fe20900033
:1062f0000100e000010032003b003700640147006c
:106300000000200001f823000089be00640147005e
:106310000000200001f823002001980031019800be
:10632000640147000000200001f8230040019800ac
:1063300051019800640147000000200001f823008b
:1063400060019800710198002c003700640147003b
:10635000a0ff2f00f18923000089be0064014700df
:10636000a0ff2f00f189230020019800310198003f
:1063700064014700a0ff2f00f1892300400198002d
:106380005101980064014700a0ff2f00f18923000c
:1063900060019800710198001800370064014700ff
:1063a000a0322300f19f23000089be006401470052
:1063b00090ff2f00f19323002001980031019800f5
:1063c00064014700a0322300f19f230040019800a0
:1063d000510198006401470090ff2f00f1932300c2
:1063e00060019800710198000200200003f82b0062
:1063f00052279800632798008f003700ae11900055
:10640000032f98000e289000e10f50002b0032005f
:106410008e289000e18f500004003c000e2990006f
:106420000200e000080032007b0037008e29900057
:10643000e28f51003e0032000e289000e30f500022
:1064400058003200740037002e109000e40047001e
:106450004200dd00010040001001be00322798001c
:10646000432798003e109000cf80de0042f20700e4
:1064700010279800212798003e1090000000e000af
:1064800007003d0002002000037824001e20900039
:10649000ae20900064f20700102798002127980092
:1064a0001e219000ae2190003e209000ce20900052
:1064b000baf20700008fbe005c0037002e1090007b
:1064c000e40047004200dd00010040001001be0072
:1064d000721f9800032798003e109000cf80de00c6
:1064e00025f20700501f9800611f98003e10900091
:1064f0000000e00007003d000200200003782400b7
:106500005e189000ee18900047f20700501f9800a8
:10651000611f98005e199000ee1990007e1890009f
:106520008e2090009df20700008fbe003f003700d4
:106530002e109000e40047004200dd000100400002
:106540001001be00321f9800431f98003e109000bb
:10655000cf80de0008f20700101f9800211f98006e
:106560003e1090000000e00007003d000200200007
:10657000037824001e189000ae1890002af207003d
:10658000101f9800211f98001e199000ae1990004e
:106590003e189000ce18900080f20700008fbe00d9
:1065a000220037002e109000e40047004200dd007a
:1065b000010040001001be0072179800031f9800f0
:1065c0003e109000cf80de00ebf1070050179800de
:1065d000611798003e1090000000e00007003d00a9
:1065e00002002000037824005e109000ee1090005e
:1065f0000df2070050179800611798005e11900087
:10660000ee1190007e1090008e18900063f207004b
:10661000008fbe00050037000000200001f82b00ad
:106620005027980061279800030037001e01be0024
:1066300052279800632798005e209000ee2090007b
:106640000080fa00000006000800fa00881f7800a9
:1066500010079800210798000000eb00000f780059
:106660001e009000104078000004e00003003a0093
:106670000000eb0030079800460037001e0078004d
:10668000800078002e0090000080400010407800cc
:106690000000fb0061e80700000478001e0078009d
:1066a000800078001e0090000080400010407800bc
:1066b0000000fb0059e80700800f5400150032006d
:1066c0002e0090000000e800200798002e009000a7
:1066d000104078000004e00003003a000000eb00e6
:1066e000300798002b0037002e0090009040780073
:1066f000c0c7b30080cf5000f1ff3a002e009000d9
:106700000000e800200798000000eb00000f780070
:106710001b0037001e0fe8001e0078008000780084
:106720002e00900000804000104078000004e0003f
:10673000080032001e007800800078002e009000d3
:106740000080400090407800c0c7b30080cf500068
:106750000b003a001e007800800078001e009000b8
:106760000080400010407800520007000000e00068
:1067700003003a001e00780030079800050037003b
:10678000700220009e0f1000bcff34001e00780035
:10679000300798003e0090004f0478000080fa0017
:1067a000000006000600fa00100798002107980074
:1067b0000080eb00000f78000e0037001e009000f4
:1067c000104178001e007800800078002e009000b4
:1067d0000080400010407800804f510005003a00d2
:1067e0001e0090000000e800100798000080eb00f9
:1067f000000f78001e0fe8001e007800800078006f
:106800002e00900000804000104078000004e0005e
:10681000eaff3a001e0090000080fa000000060027
:106820000400fa00000f780081252a001e0078007d
:10683000dcff0700000f78001e0078009040780011
:10684000d0c2b30080cf5000050032001e00780097
:1068500090407800b0c2b30080cf500001003a00f1
:106860001e0fe800b1252a001e007800cdff0700aa
:10687000000f7800d1252a001e007800c9ff07000c
:10688000000f78001e007800104078000004e0003f
:10689000030032000000eb001007980002003700f0
:1068a00010002000100798001e0090000080fa00e1
:1068b000000006000400fa00004f78001e00fb00f4
:1068c000dde707000000e00003003a00f0c5b30078
:1068d0009e4f100003003a0010002000100798009f
:1068e000020037000000eb00100798001e00900027
:1068f0000080fa00000006000c00fa002007980053
:1069000031079800420798000000eb00000f780064
:1069100081252a002e009000a2ff07002007980082
:106920001e0037001e0078004200dd008000780065
:106930003e00900000804000900078002e00900003
:1069400041ff0700100798001e0090000000e000c3
:10695000110032001e009000800078002e00900090
:106960000080400081252a008eff07002007980044
:106970001e0078004200dd00800078003e0090009c
:1069800000804000900090002e0090000100010067
:10699000500798000c0037001e0fe8001e0078001a
:1069a0004200dd00800078003e0090000080400042
:1069b00010007800104078000004e000d9ff3a0091
:1069c0004e009000500798005e0090000080fa0092
:1069d000000006000000fa000000eb0080088800bc
:1069e0000000eb0030088800f07f24006008880079
:1069f00084e0a90094e0a80011e1a8000080fa005a
:106a0000000006000000fa00b30007000080fa0052
:106a1000000006000200fa00000f78001e00780057
:106a2000100078000080fa00000006000200fa0062
:106a3000000f78001e007800640007001e00780038
:106a4000020007000080fa00000006000200fa00c1
:106a5000000f78001e0178006000b8003001980037
:106a600041019800960007001e017800100198006f
:106a7000210198000080fa00000006000600fa00dc
:106a8000200798008e000700008fbe002e009000a7
:106a9000100078000000e000230032002e0090007b
:106aa000a000900010009000be0f5000ae8f580064
:106ab0000f0036002e00900030019000c0019000c1
:106ac0002e009000a0009000100090003e024000b8
:106ad000ae8248000400be000200400083804800ef
:106ae0002e01900030019800410198000e003700ff
:106af0002e00900030019000c00190002e00900008
:106b0000a0009000100090003e021000ae8218001d
:106b10000400be0002004000838048002e01900067
:106b200030019800410198002e0090001e01be0027
:106b300012009800230098002e009000300390006f
:106b4000c003900086007800a0002000000ab80072
:106b50006030b90005017800000141006a38b900d1
:106b600000014100820278000400be000080fa00ab
:106b7000000006000200fa00000f78001e007800f6
:106b8000beff07009e0078001000200080087800fb
:106b90001e00780030039000c0039000860078004b
:106ba000a0002000000ab8006030b900050178009c
:106bb000000141006a38b9000001410082027800fa
:106bc0000400be000080fa00000006000200fa0087
:106bd000000f78001e007800a8ff07009e007800d4
:106be0000000eb00800878001e0078003003900061
:106bf000c003900086007800a0002000000ab800c2
:106c00006030b90005017800000141006a38b90020
:106c100000014100820278000400be000080fa00fa
:106c2000000006000600fa00200798002400070074
:106c30000001be002e00900001002000001f410056
:106c4000019749001e000700be0f5000ae8f58008c
:106c5000fcff39000080fa00000006000600fa0080
:106c60002007980016000700008fbe002e0090003d
:106c7000e90f5000080036002e009000a20020000e
:106c8000110009000280d800010020001e0f400002
:106c90005e9748000400370010002000010020002b
:106ca0001e0f40005e97480005000700be0f500011
:106cb000ae8f5800fcff39000080fa00000006008b
:106cc0000000fa0004000700d0518000e15180006c
:106cd0000080fa00000006000200fa00c2518000a5
:106ce000d0518000e1518000000f51001e0078005b
:106cf0006101b800d0518000e151800002004000e5
:106d000083804800d0518800e15188000080fa005b
:106d100000000600801f78000000fa000000eb0071
:106d200030088800c05180000000e800c051880091
:106d300084e0a9000080fa004f00780000400600bf
:106d40008800fa00416a20009140780000ccb3002e
:106d500000c060003040b300a4e6b700416c2000e2
:106d60009140780000ccb30000c060003040b30018
:106d7000c4e6b700d6f50700a8f90700d30107005d
:106d800014ff0700e4004700a0162a00801f7800c7
:106d900030172a00801f7800f0172a00801f780023
:106da000010078008ce60700e6875700e400470002
:106db0001000200052fa0700400720000e0040009b
:106dc00022ff0700400720000e00400069ff070077
:106dd000e00720000e0040001cff0700e007200035
:106de0000e00400063ff070000003700400720004e
:106df0000e00400021ff07000001be00803e200081
:106e000001002000800f5100818f590001003600e1
:106e100000000000e00720000e00400017ff070000
:106e20000001be004006200001002000800f51003c
:106e3000818f590003003600e00720000e0040005b
:106e400002ff0700640047002e0007000000e0007a
:106e500003003a00300020001007980010003700af
:106e600064004700211c2a004efe0700000f780036
:106e70001e007800104078000004e00003003a0093
:106e80002000200010079800050037004200200075
:106e9000611f2a001e00780097fe07001007980067
:106ea0001e009000e30f5000d0ff32001e00900043
:106eb0000000e0000f0032001e009000e20f5000c2
:106ec0000c003200400520000e0040009e009000a3
:106ed000811f7800511c2a00811f78003ee60700c0
:106ee000e4875700410520008e80400010002000fc
:106ef00003fa0700011d2a001000200000fa070015
:106f0000baff37000800fa00300798000000eb00d5
:106f100010079800e4004700100020009ff90700c8
:106f20000000e0003f003200ce4090001000200042
:106f3000bbf907004e409000ed4f500003003a00af
:106f4000a1c0b30010002000b5f907004e4090002a
:106f5000ed4f50001a0032004e409000e84f5000b4
:106f60000d00320001528000f0042000808f50009c
:106f700009003c00025280004e40900080407800a2
:106f8000809a200000004100014878000200e800db
:106f90000052880006003700005280000000e00028
:106fa00003003400005280000000e9000052880015
:106fb000be0090000040eb008048780019003700c8
:106fc000100020001007980001528000809a2000d5
:106fd000808040000040eb00804878000000eb001b
:106fe000000f78000a0037001e007800800078004b
:106ff0003e009000008140009e007800809a2000b2
:107000000080400010407800004978001e0fe80022
:10701000005280009e0f1000f3ff34000000eb00d0
:10702000005288001e0090000080fa000000060058
:020000040000fa
:10703000380a0000060000000000000018090000e7
:107040009000000000000000f8090000400000006f
:10705000000000003e0a00000200000000000000e6
:10706000a80900005000000002000000000000001d
:107070000000000000000000000000000000000010
:107080000000000000000000000000000000000000
:1070900000000000000000000000000000000000f0
:1070a00000000000000000000000000000000000e0
:1070b00000000000000000000000000000000000d0
:1070c00000000000000000000000000000000000c0
:1070d0000000000000000000400a00000200000064
:1070e00000000000420a0000020000000000000052
:1070f000000800001801000000000000440a000021
:107100004a000000020000000000210015110e00de
:107110000d0c0b000b0a0a000909090009090800f7
:107120000808080008080800070707000707070005
:107130000707070007070700073031003233340024
:107140003536370038396100626364006566670070
:1071500068696a006b6c6d006e6f7000717273000d
:1071600074757600777879007a000000440b00008f
:107170000400000002000000000000000000000009
:107180002a0b0000120000000200000001000200b3
:10719000000400000800100000000000202b2d005b
:1071a000233000003c0b000008000000020000003b
:1071b000686a6c00747a4c0000000000080b000044
:1071c000220000000200000030313200333435006c
:1071d000363738003961620063646500660030004c
:1071e00031323300343536003738390041424300fc
:1071f00044454600000000008e0a000048000000e0
:107200000200000000000000000000002440000018
:1072100000000000000059004000000000000000d5
:1072200088c34000000000000084d70097410000a0
:1072300080e0370079c3410043176e0005b5b50003
:10724000b8934600f5f93f00e9034f00384d32008e
:107250001d30f900487782005a3cbf00737fdd0083
:107260004f157500d60a0000320000000200000031
:107270004e414e00006e61006e0049004e46000017
:10728000696e660000303100323334003536370025
:107290003839610062636400656600003031320095
:1072a0003334350036373800394142004344450015
:1072b00046000000480b0000020000000200000031
:1072c000000000004a0b0000020000000200000065
:1072d000300000004c0b0000020000000200000023
:0872e0000000000000000000a6
:020000040000fa
:1072e8000600fa00004f7800110798001e00900071
:1072f800440007000000e000030032000000eb003b
:1073080020079800100037001e00900090007800b9
:107318001e00900010009000008040001e48780079
:107328001e009000100090008000e8001e009000f1
:1073380030009000808060001e00900011009800ce
:1073480010002000200798002e0090000080fa000e
:10735800000006000600fa00000f780011079800e8
:107368001e0090003b0007000000e000060032000d
:107378009e0078000040eb00804878000000eb0099
:1073880020079800120037001e0090009000780037
:107398001e0090002000900000804000904078007f
:1073a8001e007800014878001e0090002000900020
:1073b8008000e8001e00900030009000808060008f
:1073c8001e0090002100980010002000200798005f
:1073d8002e0090000080fa00000006000200fa006b
:1073e800000f78009e0078000000eb00a0009800d5
:1073f8009e0078000000eb00900098000080fa00e2
:10740800000006000400fa00000f78001e00780053
:10741800100090008000e8001e0078003000900006
:10742800808060001e00780020009000808f50004f
:1074380003003a00100020001007980002003700ef
:107448000000eb00100798001e0090000080fa0072
:10745800000006000400fa00000f78001e00780003
:10746800a00090001e00780010009000808f50004f
:1074780003003a00100020001007980002003700af
:107488000000eb00100798001e0090000080fa0032
:10749800000006000200fa00000f78001e007800c5
:1074a800900090001e00780020009000808050001e
:1074b8001e00780030009000008060000080fa0014
:1074c800000006000000fa006382a9006362a900b8
:1074d8006342a9006322a8006302a90062e2a9002e
:1074e80062c2a90062a2a80021262000914078006b
:1074f80030ceb30000c0600062e2b70062c2bf00d5
:107508003040b30062e2b70065e2a90065c2a90095
:1075180065a2a9006422a9006402a90061e2a8008a
:10752800811f7800821f7800831f78002174200053
:1075380062042000730520008248780083487800a0
:1075480042c7a900cf0178004f017800cf0078002a
:10755800c16a20009140780000ccb30000c06000f0
:10756800d040b300ace6b700c16d20009140780070
:1075780000ccb30000c06000a040b300dce6b70058
:10758800216d20009140780000ccb30000c060005d
:10759800b040b300d2e6b700811f7800821f7800a0
:1075a800831f7800217420006204200073052000e6
:1075b800824878008348780042c7a800cf01780045
:1075c8004f017800cf0078000080fa000000060024
:1075d8000200fa00000f78001e00780040138800af
:1075e80060c2bf00614060000004e000fcff3200a0
:1075f8000000eb00000f7800401380000080fa00c4
:10760800000006000000fa00105280000000e000b0
:1076180001003a00ff3ffc00105280000000e80023
:10762800105288000080fa00000006000000fa00ee
:10763800105280000000e9001052880010528000ab
:107648000000e00001003a000000fc000080fa00a1
:047658000000060028
:020000040000fa
:04765c000000fe002c
:00000001FF
